:020000000628D0
:080008000B110900831685109D
:10001000061283120130003C03192628053099008E
:1000200001309A0080309B0085200230A100B4206E
:100030000530970001309800762006160130A100A7
:10004000B42006120130A100B4200A280D088F0048
:100050006E308E0000000000000000000000000074
:100060008E0B2A288F0B2828080011088C00D03E00
:1000700000300318013E8A000C08CF2094001108BC
:100080008C00D93E00300318013E8A000C08D820AD
:10009000950010088400000814048000FF309300CD
:1000A0001308003C0130031900019303003C0319BD
:1000B0005A285028093096000310031C64280008B1
:1000C0001404800003186728000815058000863096
:1000D0009300930B69280000920C960B5D28000892
:1000E0001404800001308D002620080017089000BD
:1000F0001808910055309200352017089000180814
:1001000091000030920035200800190890001A086C
:100110009100553092003520190890001A0891007E
:10012000033092003520190890001A0891001B082E
:100130009200352008001C0890001D0891005530E1
:10014000920035201C0890001D089100013092009B
:10015000352008001E089F001430A0000000000099
:10016000A00BAE289F0BAC282108003C01300319DE
:100170000001003C0319CE280030A2000A30220200
:10018000013003180001003C0319CB2864308D00B6
:100190002620A20ABE282108A103B428080082074D
:1001A00001340234043408341034203440348034B0
:1001B0008207FE34FD34FB34F734EF34DF34BF34D0
:0201C0007F348A
:00000001FF
